:1000000000308A00172800002230840000080319FD
:1000100016280630F800F701F70B0C28F80B0B2810
:100020007B30F700F70B1228800B0928003484017D
:100030001F30830583161F149F141F159F1107304F
:100040009C00FF308312A00083161F149F141F15FD
:100050009F1183121F109412A0122008831687008C
:10006000831220162008831687008312A01120080F
:1000700083168700003083129400831694000108D1
:10008000C73908388100831290010030F8009200CF
:1000900000308316920007309C0005081030F700EE
:1000A000F70B502800001C0883120D1383169D01C6
:1000B00002308312A100FA30A2000420A10B5B28B9
:1000C00083168610831286140230A100FA30A20033
:1000D0000420A10B662883168610831286108316CF
:0400E0005828630039
:02400E003A3F37
:00000001FF
